:100000000C9409010C9426010C9426010C942601F1
:100010000C9426010C9426010C9426010C942601C4
:100020000C9426010C9426010C9461110C94351249
:100030000C944A0C0C9426010C9426010C94260175
:100040000C9426010C9426010C9426010C94260194
:100050000C9426010C94D10C0C9426010C942601CE
:100060000C9426010C9426010C9426010C94260174
:100070000C9426010C9426010C9426010C94260164
:100080000C9426010C9426010C9426010C94260154
:100090000C9426010C9426010C9426010C94260144
:1000A0000C9426010C9426010C942601075A095A37
:1000B0000B5A0D5A115A1A5A1C5A1E5A205A225AB1
:1000C000085A0A5A0C5A0E5A125A1B5A1D5A1F5ACB
:1000D000215A295A015A015A0F5A105A015A185ACC
:1000E000195A015A015A015A00D0D0D0D0D0D001AB
:1000F00001020408102041424448480000004848DA
:1001000050608182848890A0C1C2C4D0D0D0D0D0A9
:10011000D0C8000000000000000000000000000047
:1001200000000000000000001003470068006500A8
:1001300072006B0069006E00000020033400300084
:100140002000500065007200630065006E007400BE
:10015000200043006C0075006200000004030904E5
:1001600009025F00030100A0FA0904000001030175
:100170000100092111010001224000070581030847
:100180000001080B01020202010009040100010242
:1001900002010005240010010424020205240601C6
:1001A00002070582030800FF09040200020A00009A
:1001B0000007050402100005070583021000051260
:1001C000010002EF02010825406060010001020009
:1001D0000105010906A101050719E029E715002518
:1001E00001950875018102950175088101050719BE
:1001F0000029FF150026FF009506750881000508F7
:100200001901290595057501910295017503910163
:10021000C00011241FBECFEFDAE0DEBFCDBF11E07A
:10022000A0E0B1E0E2E2FCE202C005900D92AE3344
:10023000B107D9F721E0AEE3B1E001C01D92A73AC2
:10024000B207E1F70E94F1070C9405160C94000028
:1002500081E0089581E008950E942A01089508959B
:100260000E942F010895A5E0B0E0E9E3F1E00C94CD
:100270008615FC0195E0DE01119601900D929A958C
:10028000E1F789819A810E94C20369817A810E9483
:10029000CE052596E2E00C94A21581E00895CF9357
:1002A000DF93EC0160E00E943301BE010E94300147
:1002B000DF91CF9108950E94AC0608950E94B00688
:1002C000089508950E94B0030E9461012FEF84E316
:1002D0009CE0215080409040E1F700C0000008956C
:1002E0000E9462010E94F50C08950E9462010E9422
:1002F000060D08950F931F93CF93DF93EC0161E0F8
:100300000E9433018C01BE010E942C01811106C0A4
:1003100080E0DF91CF911F910F910895BE01C80138
:100320000E945C088823A1F3BE01C8010E94220B31
:10033000882371F3BE01C8010E942609882341F376
:10034000BE01C8010E94940A882311F38A81882380
:1003500099F00F3D8CE5180751F0083A8DE5180724
:1003600041F001151C4541F40E947001D1CF0E945B
:10037000E8040E947501CCCFCE010E942801C9CFAC
:100380000E94270C0E94010208950E9405020E940B
:100390002C0C0895292F332740E02115310511F049
:1003A000C90148E09C0164E0369527956A95E1F71C
:1003B0002115310511F04C5FC9019C013695279537
:1003C000369527952115310511F04E5FC901969597
:1003D0008795892B09F04F5F842F089508950E9417
:1003E000EE01089581E008950E94F20108950895B4
:1003F000CF93C82F0E94EF018C2F0E94F401CF9160
:10040000089580E00E94F80108950E947E0B0E94EA
:10041000F8010895CF930E947E0BC82F8091400170
:100420008C1779F0C09340010E94B60C6093410193
:100430007093420180934301909344018C2F0E945A
:10044000F801CF910895CF93C82F8823C9F082383F
:10045000C9F40E947E0B81FD13C089E30E94D8037A
:100460000E94EF032FEF87EE93E0215080409040F1
:10047000E1F700C0000089E30E94E0030E94EF035F
:10048000CF9108958338A1F40E947E0B80FDF8CFB0
:1004900083E50E94D8030E94EF032FEF81EE94E0E2
:1004A000215080409040E1F700C0000083E5E4CF98
:1004B0008438A1F40E947E0B82FDE2CF87E40E9483
:1004C000D8030E94EF032FEF81EE94E0215080408B
:1004D0009040E1F700C0000087E4CECF8CEF8C0F96
:1004E000813A90F46C2F80910001909101010E945B
:1004F000C20B882329F08C2F0E94E0030E94EF0397
:100500008C2F0E94D803BACF80E28C0F883008F07D
:10051000B7CFC77081E001C0880FCA95EAF70E9483
:100520001F04ACCF882309F44DC0823879F40E94AF
:100530007E0B81FF47C089E30E94D8030E94EF032E
:1005400089E30E94E0030E94EF030895833859F481
:100550000E947E0B80FF36C083E50E94D8030E9474
:10056000EF0383E5EECF843859F40E947E0B82FFBF
:1005700029C087E40E94D8030E94EF0387E4E1CFFB
:100580009CEF980F913AE8F290E2980F983050F46F
:10059000877091E001C0990F8A95EAF7892F0E9430
:1005A0002504D1CF9BE5980F933028F490E080E0AC
:1005B0000E94960B0895885A873120F490E080E0DD
:1005C0000E94AC0B0895CF93DF93D62F7032D0F4F6
:1005D000C72FCF70707F11F0C295C07FFC01828160
:1005E0008823B9F0CC2359F080E28D0F883010F0C9
:1005F000D1110BC08C2F0E941F040E94EF038D2F7E
:100600000E942302DF91CF9108958C2F0E942F0426
:10061000F4CF8D2F0E949202CC23A1F380E28D0FA4
:10062000883010F0D11106C08C2F0E9425040E9442
:10063000EF03E8CF8C2F0E943504F9CFCF93DF93DF
:10064000EC01688179818A810E94D403BC01CE01CA
:100650000E94E302DF91CF910895CF93DF93EC01E5
:100660008B819C81892B29F08881998189238F3FF7
:1006700019F4DF91CF910895CE010E947A01882369
:10068000C1F3CE010E941E03CE010E944F01F1CFA3
:10069000AAE0B0E0EEE4F3E00C9486154E835F83AD
:1006A000688779878A8761110E943C0485E0FE0192
:1006B0003696DE01119601900D928A95E1F78C81B4
:1006C0009D81892B41F4CE0101960E942D032A962B
:1006D000E2E00C94A21589819A8189238F3F99F3D6
:1006E000CE0101960E944D018111EDCFF0CF1F93F5
:1006F000CF93DF93182FEB010E942302209739F448
:10070000812F0E949202DF91CF911F9108958FE96E
:100710009FE00197F1F700C000002197EFCF70E054
:1007200060E0893311F460E570E00E94770308957A
:10073000882321F00E941F040E94EF03089588235C
:1007400021F00E9425040E94EF0308950E943C04BA
:100750000E94EF0308950E94E8030E94A6030895F3
:100760000E942C040E94AB03089508950E94B503D3
:1007700008950E94B60390934601809345010E941C
:10078000A603089580914501909146010E94CA01F7
:100790000895CF93DF93EC010E94C203BE010E9433
:1007A000E905DF91CF910895CB010E94C903089517
:1007B000682F80910001909101010E94F80B08952B
:1007C000682F80910001909101010E94FB0B089518
:1007D00080910001909101010E94FE0B0895CF933A
:1007E000DF93E0910001F091010180915801808335
:1007F000E0910001F0910101808190915701892BD6
:100800008083C0910001D091010148E050E067E48D
:1008100071E0CE010E94AD15892B59F088E0FE01F0
:10082000A7E4B1E001900D928A95E1F7CE010E9414
:100830008B0BDF91CF91089580915801089590918D
:100840005801892B80935801089580959091580103
:10085000982390935801089510925801089590910B
:100860005701892B809357010895809590915701E6
:10087000982390935701089510925701089590E09E
:1008800080E00E94CB1521E0883E9E4F09F020E0D9
:10089000822F089582E090E00E94C315089583E0BE
:1008A00090E00E94C3150895CF9384E090E00E94E9
:1008B000C315C82F82E290E00E94C315982F8C2F99
:1008C000CF910895CF93C92F682F84E090E00E94C4
:1008D000D1156C2F82E290E00E94D115CF9108953E
:1008E000AB01BC018FE090E00E94E3150895AB01DD
:1008F000BC0183E190E00E94E315089560E070E0A0
:10090000CB010E947704089560E070E0CB010E9463
:1009100070040E947E04089568EE7EEF90E080E00F
:100920000E94EF1560E082E090E00E94D11560E047
:1009300083E090E00E94D11510924601109245018B
:1009400060E084E090E00E94D11564E082E290E0F3
:100950000E94D11560E085E090E00E94D11560E032
:1009600086E090E00E94D1156FEF87E090E00E9452
:10097000D11540E050E0BA0188E090E00E94E31514
:1009800060E08DE090E00E94D11540E050E0BA01B7
:1009900088E190E00E94E31560E087E190E00E942A
:1009A000D11540E050E0BA018CE190E00E94E315DF
:1009B00070E060E080E290E00E94EF1540E050E0DF
:1009C000BA0188E190E00E94E3150E948404089532
:1009D0000E948C040895682F8EE090E00E94D1154B
:1009E00008950E94B60C6093640170936501809332
:1009F0006601909367016093600170936101809339
:100A00006201909363010895089508950E94050579
:100A1000089508950E940905089580E996E00E94CE
:100A2000740B0E9404050E940605089581E0089554
:100A30000E9416050895089508950E941B050E94BE
:100A40001C0508950E9493060E94F70108950E94D4
:100A5000A10C0E9454070E9422050E943C080E949B
:100A60004C0E0E940A050895AAE0B0E0EAE3F5E022
:100A70000C947E150E946A078BE5A82E81E0B82EA3
:100A8000750110E0F70101917F01812F0E94B306EB
:100A90001F5F153009F440C00817A1F38091680169
:100AA00081FD0E94B9060E941805C82E10E0812F12
:100AB0000E94B306082FF50181915F01081731F1FB
:100AC000D02ED826F12CEE24E3948D2D8E21B1F07A
:100AD000CC20A1F0FE821F8391E0802F8E2109F4AB
:100AE00090E098870E94AA0C8160782F9A87898766
:100AF0004E815F8168858A850E944803F394EE0CDD
:100B0000F6E0FF12E2CFF501319700831F5F153049
:100B100071F60E94F10420C00813C0CF0E94AA0CF5
:100B20008C018091590190915A0108171907A1F081
:100B30008FEF89838A831B820E94AA0C8160782FA1
:100B40009D838C8349815A816B818D810E944803EA
:100B500010935A01009359010E940A022A96EAE072
:100B60000C949A150E94EE05883E910588F4803E0B
:100B7000910598F48130910581F0009771F09C0106
:100B800024503109213A310540F090E080E005C061
:100B90009C013A9521153F41C0F70895972F753074
:100BA000A8F4663098F470E026E0929F600D711D05
:100BB0001124FB019EE1899FE00DF11D1124EE0F30
:100BC000FF1FE455FF4F85919491089580E090E0D8
:100BD00008950E94CE050E94B205089582389105BD
:100BE000B9F1B0F48133910509F47DC048F489323C
:100BF000910509F46DC08A32910509F47BC008950E
:100C00008533910509F45FC08933910509F1089591
:100C1000833E9105D9F138F4803E910529F1823E59
:100C2000910579F10895863E9105D9F1873E9105A8
:100C300009F43EC0843E910541F520918B0121FFCE
:100C400024C080918A0184FD19C087EE90E0089548
:100C500020918A01237009F05AC020918B0123FF53
:100C600014C089E290E0089520918A0120FD38C0E7
:100C700030918B0130FF09C024FF43C090E080E039
:100C8000089520918A0122FDF7CF089520918A01CD
:100C900022FD3AC030918B0130FD39C024FFF5CFE1
:100CA000EDCF20918A0123FFF0CF24FDE7CFCDCFF8
:100CB00020918A0123FD2EC030918B0131FFEECFB0
:100CC00084EE90E0089520918A0125FFDECFC9CF00
:100CD00020918A0125FD21C020918B0123FFD5CFD2
:100CE00089E390E0D2CF20918A0126FFCECF8AE21D
:100CF00090E0089520918A0126FFC7CF81E390E01C
:100D0000089583EE90E0089582EE90E0089580EEDD
:100D100090E0089586EE90E0089585E390E00895D0
:100D200080E0089508950E943F04811102C00E944E
:100D3000E8040E944A04809368010E94540490933E
:100D40008B0180938A010E9492060E944F0490E0DA
:100D50000E94B903089508950E94AB06089508956E
:100D60000E94AF060895E82FF0E0EF56FE4F808115
:100D70000895089580EA8A95F1F7089500C00895CE
:100D80000E94BA060895F894E82FE295EF70F0E01B
:100D900031A1282F2F7081E090E001C0880F2A95A3
:100DA000EAF7982F9095932391A392A1892B82A380
:100DB00078940895CF93DF93C8E3D1E089918F3F72
:100DC00011F00E94C30681E0CD33D807B9F7C2E322
:100DD000D1E089918F3F11F00E94C30681E0C833B2
:100DE000D807B9F7DF91CF910895B0E0A0E0EBEF1D
:100DF000F6E00C948015EC01D62E062F10E0C80109
:100E0000885C9E4F7C01FC0180818F3F09F445C0C6
:100E1000F894E82FE295EF70F0E091A18F7021E057
:100E200030E001C0220F8A95EAF7892F822B81A337
:100E300082A12095282322A378940E94BE06E2E393
:100E4000F1E048E351E031E0C12C21912F3F51F115
:100E5000A22FA295AF70B0E090968C9190E02F7089
:100E600002C0959587952A95E2F780FD1BC0832FD8
:100E7000C82A330F4E175F0741F7F70180818F3F74
:100E800011F00E94C30661E0C11001C060E08D2D29
:100E90000E94C006C00FD11FC882CDB7DEB7E8E000
:100EA0000C949C1580E0E4CF0E94DA0685E0E1E92D
:100EB000F1E0DF01982F1D929A95E9F7ECE8F1E057
:100EC000DF011D928A95E9F785E00E94A5070E943F
:100ED0005B010895A5E0B0E0E0E7F7E00C9483152E
:100EE0008E010F5F1F4F85E0F80111928A95E9F797
:100EF000F12C6F2DC8010E94F506F394F5E0FF1266
:100F0000F8CF45E050E0B8018CE891E00E94AD15C3
:100F100021E0009709F420E0892B41F085E0F801F9
:100F2000ACE8B1E001900D928A95E1F745E061E906
:100F300071E08CE891E00E94A607182F0E945E01E4
:100F4000812F2596E5E00C949F150895CF92DF92AE
:100F5000EF92FF920F931F93CF936C017B01042FAD
:100F6000222349F081E080936B010E94AA0C9093A8
:100F70006A0180936901C0916B01C1110AC0C0E090
:100F80008C2FCF911F910F91FF90EF90DF90CF901A
:100F900008958091690190916A010E94C20C0597A1
:100FA00070F310E0A801B601C7010E94AD15892BAE
:100FB00041F0A801B601C7010E94BA1510926B0159
:100FC000DFCFC0E0FBCF0E94C30E0E9427050E9426
:100FD000D00E08950E94D50E0E9434050E94EF0E97
:100FE00008950E94430C0E94A90E0E940D050E94C4
:100FF000E3070E94EA070E941D05FBCFEEE6F1E041
:1010000086E0DF011D928A95E9F70895CF93DF937B
:1010100080916E01806880936E01CEE6D1E0899167
:101020000E946C0E81E0C437D807C9F7DF91CF91D9
:101030000895282F67E00E94641590E0FC01E259B2
:10104000FE4FAC0133E0440F551F3A95E1F7841B86
:10105000950B820F911D26E030E0281B390B81E0B3
:1010600090E0AC0102C0440F551F2A95E2F7808141
:10107000842B808380E008950E943F04811102C088
:101080000E94E8048DE090E00E94C31580936C01FB
:101090000895CF93C82F0E94FE07C0936C016C2F58
:1010A0008DE090E00E94D115CF91089581E00895E0
:1010B00081E0089581E00895EF92FF920F931F93CE
:1010C000CF93DF937C01EB018C011A55003411059D
:1010D00050F48B819C81892B31F0888199818923FF
:1010E0008F3F09F0A0C0C1E057C081E3E8168AE550
:1010F000F80609F0A9C08B819C81892B09F4A4C052
:101100008881998189238F3F09F49EC08A81882331
:1011100009F49AC080E010C08B819C81892B09F46E
:1011200093C08981988189238F3F09F48DC08A817A
:10113000882309F489C081E00E94490885C0009194
:101140006D0110916C018B819C81892B31F088811C
:10115000998189238F3F09F043C0015000936D01AD
:101160002EE631E0412FBE01C7010E9458088823B6
:1011700009F46AC080916D0118160CF465C01092D4
:101180006D016EE671E080916C010E945608C82FD7
:1011900081110CC00E94FE078C2FCDB7DEB7E6E0B0
:1011A0000C949E158E2D0E94190835C080916C01FB
:1011B000882399F0813071F4CEE6D1E002E711E0A6
:1011C000899181110E946C0E0C171D07C9F780E0F0
:1011D0000E946C0E0E94FE0737C00E940608FACFDC
:1011E0008A81882309F4B9CF0F5F00936D01112321
:1011F000C9F2113049F5F701FF27E851FF4FE4919B
:10120000AE2FA295A695A695A370B0E0A259BE4FA9
:101210008C91E82BEC932EE631E0412FBE01C70103
:101220000E94580811C0C7010E945A08882361F023
:1012300080E3E8168AE5F80609F46ECF08F055CF8A
:101240000A32110508F47BCFC0E0A6CFCF93DF931D
:10125000EC01FB018281882309F464C1C430FDE5FF
:10126000DF07E0F5CB3F9CE5D90730F49E01225023
:101270003C4524313105D8F50E94540490938B01EC
:1012800080938A01C231ECE5DE0709F41FC108F042
:101290006EC0C9308CE5D80709F4F2C008F03FC031
:1012A000C530ECE5DE0709F4DBC058F5C3308CE54A
:1012B000D80709F4CDC008F0CFC080918A018160C1
:1012C000C230DC4509F4AEC080918A0190918B0157
:1012D0000E9462040E94B00380E009C0C63AEDE5B6
:1012E000DE0751F238F4C2369DE5D90729F2DF91C5
:1012F000CF9108959E012E5A3D4523303105B8F710
:10130000BBCF80918A018062C730FCE5DF0709F41A
:1013100089C008F4B1C080918A01806483C0CD3057
:101320009CE5D90709F4BAC070F480918A018E7FD8
:10133000CB30FCE5DF0709F475C008F4A7C0809145
:101340008A018D7F6FC0CF309CE5D90709F4B6C004
:1013500008F4A8C0C031FCE5DF0709F4B3C0C1310F
:10136000DC4509F0B1CF80918A018F7B5BC0C1154C
:101370009DE5D90709F4B4C098F5CB3FFCE5DF073C
:1013800009F472C0B8F4C4319CE5D90709F4B6C0B9
:1013900008F4A2C0C531DC4509F096CF80918A01DE
:1013A00082FB992790F921E0922790FB82F990FB2C
:1013B00083F938C0CD3F8CE5D80709F477C008F42D
:1013C00057C0CE3FECE5DE0709F474C080918B0175
:1013D0008360CF3FDC4509F077CF80938B0174CFDA
:1013E000C2368DE5D80709F496C068F4C230EDE541
:1013F000DE0709F48CC008F477C0C330DD4509F07E
:1014000063CF80E085C0CE3A9DE5D907E9F068F466
:1014100090918A01892F8E7F90FF8160C63ADD45C9
:1014200009F052CF80938A014FCFCF3A8DE5D8078C
:1014300089F1C03BDD4509F047CF90918B01892FA1
:10144000877F93FF8860C9CF80918B018860C5CF6B
:1014500080918A018260E6CF80918A018460E2CF28
:1014600080918A018860DECF80918B018160B5CF49
:1014700080918B018260B1CF80918A018061D2CF4F
:101480000E94B00380918A018068CCCF80918A014C
:101490008C60C8CF80918B01877F9FCF80918A011C
:1014A0008B7FC0CF80918A01877FBCCF80918B01D9
:1014B0008E7F93CF80918B018D7F8FCF80918A011A
:1014C0008F7EB0CF80918A018F7DACCF0E94B00318
:1014D00080918A018F77A6CF80918A01837FA2CFE6
:1014E00080918B018C7F79CF80918B01982F909583
:1014F00091708E7F892B90FB81F96FCF0E94B00392
:1015000090918A01892F97FB87F980588BCF81E0D2
:101510000E94EB04D9CE90918A01892F8F7E94FF8F
:10152000806180CF81E0E3CECF93DF93EB01863102
:101530009C4511F50E941C049A81992399F08A7A9E
:1015400091E009F490E090937401811109C089E25F
:101550000E94D8030E94EF0380E0DF91CF910895AD
:1015600085E3F6CF80917401811104C089E20E9465
:10157000E003F0CF85E3FBCF81E0EFCF0F931F9324
:10158000CF93DF93C42FD22FFC0182818823C9F02F
:10159000409377010E94AA0C909376018093750185
:1015A00080E28C0F883040F4C77081E001C0880F62
:1015B000CA95EAF70E949803DF91CF911F910F918E
:1015C000089510917701141332C0809175019091A4
:1015D00076010E94C20C883C910548F5C0E2CD0F0F
:1015E0001D17B9F080E2810F883040F4177081E058
:1015F00001C0880F1A95EAF70E949F03C83048F48B
:1016000081E09D2F977001C0880F9A95EAF70E949C
:101610009803802F0E948F03C83070F6D77081E046
:1016200001C0880FDA95EAF70E949F03C5CF80E2D8
:101630008C0F883008F6C77081E001C0880FCA950A
:10164000EAF7F2CF0F939C01CB01243F4CE534071E
:1016500059F1A8F4293DFCE53F0701F12A3D4CE58D
:101660003407D1F1283D3C4591F406E221EE41EEEC
:1016700068ED7CE50E94BE0A80E00F910895263F48
:10168000FCE53F07E9F0B0F0273F3C45F9F0FC01ED
:101690008281882339F110927701EFCF07E225EE9E
:1016A00045EE69ED7CE5E6CF06E221EE40EE64EF23
:1016B0007CE5E0CF07E225EE44EE65EF7CE5DACF8E
:1016C00006E221EE42EE66EF7CE5D4CF07E225EE9E
:1016D00046EE67EF7CE5CECF08E221E045EE6AED0D
:1016E0007CE5C8CF81E0C9CF90933F0180933E0154
:1016F000089590937D0180937C010895E0917C0191
:10170000F0917D01309729F00190F081E02D09954D
:10171000089580E00895E0917C01F0917D0130977B
:1017200021F00280F381E02D0995089520917A013E
:1017300030917B012817390771F090937B018093DA
:101740007A01E0917C01F0917D01309721F00680D3
:10175000F781E02D09950895209178013091790164
:101760002817390771F09093790180937801E091FF
:101770007C01F0917D01309721F00084F185E02D0E
:1017800009950895662349F0FC0132960896219147
:10179000261729F0E817F907D1F780E0089581E0CE
:1017A00008959C01FC0132969FEF80E0419146171D
:1017B00051F09F3F19F4411101C0982F8F5F86307F
:1017C000A9F79F3F09F40895290F311D97FD3A9518
:1017D000F90162830895FC0132960896219126133F
:1017E00003C0DF0111971C92E817F907B9F70895B4
:1017F0000E94D10B08950E94EB0B0895029626E0FB
:10180000FC0111922A95E9F7089508950E94050CAC
:101810000895811106C081E080937E010E94060C2C
:10182000089582E0F9CF83E080937E010E94060C48
:1018300008950E94090C089581E080937E010E9422
:10184000060C08950E941C0C0895089508950E94A6
:10185000260C0895089508950E94250C0895CF93AD
:101860000E942A0C0E946A070E942B0CC0E08C2F59
:101870000E94B306811105C0CF5FC530C1F7CF917B
:10188000089581E0FCCF85B7806885BF85B7806803
:1018900085BF08951F921FB61F9211248F939F93A7
:1018A000AF93BF9380917F01811113C08091960106
:1018B00090919701A0919801B09199014196A11D35
:1018C000B11D8093960190939701A0939801B093D6
:1018D0009901BF91AF919F918F911F901FBE1F9053
:1018E000189580919E01843031F10E94C0011092C0
:1018F0007F0188E190E020E40FB6F894A8958093EA
:1019000060000FBE2093600083B7817F846083BF37
:1019100083B7816083BF7894889583B78E7F83BFB8
:101920000FB6F894A895809160008861809360005C
:10193000109260000FBE08950E94B0030E94C5017E
:10194000089582E084BD93E095BD9AEF97BD8093A2
:101950006E0008952FB7F8948091960190919701A9
:10196000A0919801B09199012FBF08952FB7F894D5
:1019700060919601709197018091980190919901E1
:101980002FBF08959C014FB7F894809196019091D4
:101990009701A0919801B09199014FBF821B930BC1
:1019A000089578941F921FB61F9211248F939F93CE
:1019B000AF93BF938091960190919701A091980168
:1019C000B09199010196A11DB11D8093960190934C
:1019D0009701A0939801B0939901BF91AF919F9106
:1019E0008F911F901FBE1F90189587E797E79093E0
:1019F00001088093000888E19AE00FB6F894A89552
:101A0000809360000FBE90936000FFCF88E19AE062
:101A10000FB6F894A895809360000FBE9093600075
:101A2000FFCF80918801089508950895CF93DF93A3
:101A3000EC0181E08093E9008FEF9091E800815004
:101A400095FD06C095ED9A95F1F700008111F5CF4F
:101A50008091E80085FF14C050E040E068E070E04D
:101A6000CE010E94550F8091E8008E778093E800A8
:101A700088E0FE01A0E8B1E001900D928A95E1F7BF
:101A8000DF91CF9108950895089580919D0181116E
:101A900009C00E94E5100E9442118091E20084601A
:101AA0008093E200089510929D0108950E941C0CFD
:101AB000089560919A0181E0611101C080E00E9467
:101AC000130C089590919E0181E0943009F080E01C
:101AD00060919A010E94190C089542E061EC81E046
:101AE0000E94611042E061EC82E00E94611042E1DC
:101AF00060E884E00E94611042E161E883E00E94B6
:101B0000611090919E0181E0943009F080E0609135
:101B10009A010E94090C08958091A001833009F474
:101B200062C050F48130D9F1823009F4A4C082E05F
:101B300091E00E94B61456C08A3009F48BC08B30F5
:101B400009F46EC0893099F780919F01813279F74D
:101B50008091A3019091A401892B49F78091E8001D
:101B6000877F8093E8008091E80082FF37C09091E2
:101B7000F3008091F200029731F48091F1008130FE
:101B800011F0863021F48091F100809388018091DA
:101B9000E8008B778093E8000E949510C8CF809171
:101BA0009F01813A21F68091E800877F8093E800C9
:101BB0008091A3019091A401892B61F468E080E8F1
:101BC00091E070E00E94A40F8091E8008B778093F1
:101BD000E800ADCF60E090E080E0F3CF80919E011F
:101BE0008111C1CF089580919F01813A09F09FCF63
:101BF0008091A3019091A401892B09F098CF809145
:101C0000E800877F8093E8008091E80080FFFCCFA8
:101C1000809129018093F1008091E8008E77BACFFE
:101C200080919F01813209F082CF8091A301909130
:101C3000A401892B09F07BCF8091E800877F8093F6
:101C4000E8000E9495108091A101809329010E94D3
:101C5000B0036DCF80919F01813209F068CF8091F0
:101C6000E800877F8093E8000E9495108091A20190
:101C7000809389015CCF80919F01813A09F057CF11
:101C80008091E800877F8093E8008091E80080FFE2
:101C9000FCCF80918901BECF82E090E09093150146
:101CA0008093140182E091E00E947A1408950895CF
:101CB000CF93DF9382E091E00E942114EC01209702
:101CC00019F4DF91CF91089582E091E00E944A14C7
:101CD0000E94570E2197F3CFCF93C091E900209136
:101CE000EC00922F917020FD90E82091120120FFCE
:101CF00012C0CF70C92B909103019F709093E9009F
:101D00009091EB0090FF04C09091EE0097FD05C00C
:101D1000CF70C093E900CF9108959FEF2091E80024
:101D2000915025FD06C025ED2A95F1F7000091118F
:101D3000F5CF8093F10082E091E00E94DC13809166
:101D4000E80080FFE5CF8091E8008E778093E8007F
:101D5000DFCF84B7877F84BF0FB6F894A8958091B2
:101D60006000886180936000109260000FBE80E880
:101D700090E00FB6F89480936100909361000FBEDD
:101D80000E94220C08950E94E5100E944211E2EE8A
:101D9000F0E080818460808378940E94C11308956C
:101DA0008DE191E00E94790B089580919E0185302C
:101DB00031F480919E01853019F00E949C0C0895A9
:101DC0000E94710C80919C01882399F30E942F0C32
:101DD000882379F30E943F0F0E94B003EACF0E944C
:101DE000580E82E091E00E940A1408950E94F90EB4
:101DF0000895292F332723303105C9F058F42130B5
:101E0000310599F122303105A9F190E080E030E010
:101E100020E01DC02132310509F122323105A9F738
:101E200080E490E021ED31E0672B79F710C099272D
:101E30008130910581F0009729F0029731F7E8E2AF
:101E4000F1E002C0ECE5F1E0849190E09F01FA013D
:101E5000318320830895EAE3F1E0F6CF89E090E052
:101E600022E731E0672B89F6F2CF82E190E02FEB99
:101E700031E0EDCF8FE590E020E631E0E8CF80E182
:101E800089BD82E189BD09B400FEFDCF8091D800F3
:101E90008F7D8093D8008091E00082608093E00085
:101EA0008091E00081FDFCCF0895AF92BF92CF9268
:101EB000DF92FF920F931F93CF93DF936C01EB019F
:101EC0008A010E94B410F82E811123C0011511055A
:101ED00039F0F80180819181C81BD90BC80ED91E39
:101EE000B12CA12C2097A9F08091E80085FD22C09B
:101EF0008091E8008E778093E80001151105A1F02C
:101F0000F80180819181A80EB91EB182A08285E07E
:101F1000F82E8F2DDF91CF911F910F91FF90DF90C1
:101F2000CF90BF90AF9008950E94B4108823D1F253
:101F3000F82EEFCFF60181916F018093F100219788
:101F4000FFEFAF1ABF0ACECFFC018091A50190919F
:101F5000A60186179707A0F06115710529F49091E5
:101F6000E8009E779093E80090E06115710551F4C8
:101F7000911108C08091E80082FF34C080E008958C
:101F8000BC01F2CF80919E018823C1F18530C1F15F
:101F90008091E80083FD30C08091E80082FDEACFA7
:101FA0008091E80080FFE1CF8091F3002091F20062
:101FB000382F6115710519F02830310558F091E07E
:101FC0002830310509F090E02091E8002E77209329
:101FD000E800CBCF81918093F100615071092F5FB0
:101FE0003F4FE7CF80919E01882341F0853041F03B
:101FF0008091E80083FFBECF81E0089582E00895DC
:1020000083E00895FC018091A5019091A6018617B7
:102010009707A0F06115710529F48091E8008E778B
:102020008093E80090E06115710551F4911108C0AA
:102030008091E80082FF35C080E00895BC01F2CFB6
:1020400080919E018823C9F18530C9F18091E80013
:1020500083FD31C08091E80082FDEACF8091E800E5
:1020600080FFE1CF8091F3002091F200382F6115BD
:10207000710519F02830310558F091E0283031050C
:1020800009F090E08091E8008E778093E800CBCF54
:1020900084918093F1003196615071092F5F3F4F19
:1020A000E6CF80919E01882341F0853041F08091F8
:1020B000E80083FFBDCF81E0089582E0089583E0CA
:1020C0000895982F973028F08F708093E90081E071
:1020D00008959093E900242F762F50E0981731F05F
:1020E0007091EC002091ED005091F00021FD02C0B4
:1020F0009F5FE8CF3091EB003E7F3093EB00309153
:10210000ED003D7F3093ED003091EB003160309376
:10211000EB007093EC002093ED005093F0002091C1
:10212000EE0027FDE5CF80E0089580919F0187FFB5
:1021300013C08091E80082FF06C08091E8008B7791
:102140008093E80004C080919E018111F2CF089530
:1021500080919E018823D9F38091E80080FFF8CF19
:102160008091E8008E77ECCF2091E4003091E5007B
:1021700095E6A9012091EC00822F817020FF06C016
:102180008091E80080FF06C080E008952091E8007B
:1021900022FD1AC080919E01882389F0853089F044
:1021A0008091EB0085FD0FC02091E4003091E500A7
:1021B00042175307F9F29150E1F684E0089582E066
:1021C000089583E0089581E008950E9454110E94CB
:1021D0005C11E0EEF0E0808181608083E8EDF0E06A
:1021E00080818F77808319BCA7EDB0E08C918E7FC2
:1021F0008C9380818F7E808310929D0108950F9330
:102200001F93CF93DF930E9454110E945C11C8ED7D
:10221000D0E088818F7788838881806888838881EF
:102220008F7D888319BC10929E0110929A011092A2
:102230009C0110929B0100EE10E0F80180818B7FE1
:10224000808388818160888342E060E080E00E9432
:102250006110E1EEF0E080818E7F8083E2EEF0E0BD
:10226000808181608083808188608083F8018081A3
:102270008E7F8083888180618883DF91CF911F91D9
:102280000F910895E8EDF0E080818F7E8083E7ED87
:10229000F0E080818160808384E082BF81E0809370
:1022A0009D010E94FF100895E8EDF0E080818E7F8F
:1022B00080831092E20008951092DA001092E100FB
:1022C00008951F920F920FB60F9211242F933F93F0
:1022D0004F935F936F937F938F939F93AF93BF932E
:1022E000EF93FF938091E10082FF0BC08091E200A9
:1022F00082FF07C08091E1008B7F8093E1000E9404
:10230000C0138091DA0080FF19C08091D80080FF4F
:1023100015C08091DA008E7F8093DA008091D90019
:1023200080FF96C080E189BD82E189BD09B400FECD
:10233000FDCF81E080939E010E94450D8091E100D8
:1023400080FF19C08091E20080FF15C08091E200FB
:102350008E7F8093E2008091E20080618093E200B2
:102360008091D80080628093D80019BC85E080936A
:102370009E010E94590D8091E10084FF2BC0809145
:10238000E20084FF27C080E189BD82E189BD89B573
:10239000982F917080FFFBCF8091D8008F7D809324
:1023A000D8008091E1008F7E8093E1008091E2006F
:1023B0008F7E8093E2008091E20081608093E20052
:1023C00080919A01882309F449C084E080939E019A
:1023D0000E94620D8091E10083FF29C08091E2009C
:1023E00083FF25C08091E100877F8093E10082E038
:1023F00080939E0110929A018091E1008E7F8093DC
:10240000E1008091E2008E7F8093E2008091E20003
:1024100080618093E20042E060E080E00E94611011
:102420008091F00088608093F0000E94560DFF912B
:10243000EF91BF91AF919F918F917F916F915F913C
:102440004F913F912F910F900FBE0F901F901895B5
:1024500019BC10929E010E94530D70CF8091E30031
:1024600087FD93E090939E01B3CF1F920F920FB61A
:102470000F9211242F933F934F935F936F937F930A
:102480008F939F93AF93BF93CF93DF93EF93FF937C
:10249000D091E900DF708091EC00C82FC17080FD01
:1024A000C0E81092E9008091F000877F8093F000EF
:1024B00078940E9479121092E9008091F00088606F
:1024C0008093F000CD2BCF70C093E900FF91EF9186
:1024D000DF91CF91BF91AF919F918F917F916F913C
:1024E0005F914F913F912F910F900FBE0F901F90D2
:1024F0001895AAE2B0E0EFE7F2E10C9485158FE9B8
:1025000091E02091F100FC012193CF01F1E0873AA5
:102510009F07B9F70E948C0D8091E80083FF1EC1D0
:1025200080919F019091A0019A3008F017C1E92F86
:10253000F0E0E95FF94E0C947015803899F082381C
:1025400009F00CC18091A3018F70873008F006C19B
:102550008093E9008091EB0085FB882780F9109239
:10256000E90006C080919B0190919C0191118260CD
:102570009091E800977F9093E8008093F10010928B
:10258000F1008091E8008E77E5C0882309F4D3C07C
:10259000823009F0E3C08091A1018111D6C0809101
:1025A000A3018F702FEF280F263008F0D7C080933B
:1025B000E9002091EB0020FFC8C0933031F48091F6
:1025C000EB0080628093EB00C0C09091EB009061C3
:1025D0009093EB0021E030E001C0220F8A95EAF7EA
:1025E0002093EA001092EA008091EB008860EACF25
:1025F0008111B4C01091A1011F778091E300807810
:10260000812B8093E3008091E800877F8093E8002E
:102610000E9495108091E80080FFFCCF8091E3003C
:1026200080688093E30082E0111183E080939E0133
:1026300095C08058823008F091C08091A10190919E
:10264000A2018C3D23E09207A1F583E08A838AE210
:1026500089834FB7F894DE01139620E03EE051E203
:10266000E32FF0E050935700E49120FF03C0E29580
:10267000EF703F5FEF708E2F90E0EA30C0F0C796AA
:102680008D939D932F5F243159F74FBF8091E800C0
:10269000877F8093E8006AE270E0CE0101960E9495
:1026A000A40F8091E8008B778093E80057C0C09614
:1026B000E7CF6091A3017091A401AE014F5F5F4F1E
:1026C0000E94F60EBC01892B09F448C09091E800E5
:1026D000977F9093E80089819A810E940210E1CF50
:1026E0008038E1F58091E800877F8093E800809151
:1026F0009A018093F10045CF811130C09091A101E2
:10270000923060F58091E800877F8093E800909395
:102710009A010E94951080919A01882311F084E01B
:1027200005C08091E30087FDFACF81E080939E0190
:102730000E946D0D13C08091A101813079F481E078
:10274000933009F080E080939C011092E900809121
:10275000E800877F8093E8000E9495108091E80050
:1027600083FF0AC08091E800877F8093E800809112
:10277000EB0080628093EB00AA96E3E00C94A11535
:102780000895CF9380919E018823A1F0C091E90024
:10279000CF709091EC00892F817090FD80E8C82B5C
:1027A0001092E9008091E80083FD0E947912CF70B9
:1027B000C093E900CF91089520919E01243041F506
:1027C000FC014489558966897789452B462B472B1F
:1027D000F9F081818F708093E9009091F3008091EE
:1027E000F200892B11F480E008959091E800809127
:1027F000E8008E778093E80095FDF5CF0E94B41035
:10280000811107C09091E8009E779093E8000895A9
:1028100082E0089520919E01243091F4FC014489C6
:10282000558966897789452B462B472B49F02181AD
:102830002F702093E9002091E80020FD0E94DC1316
:10284000089520919E01243019F090E080E00895D1
:10285000FC014489558966897789452B462B472B8E
:10286000A1F386818F708093E9008091E80082FF58
:10287000ECCF9091F3008091F200009731F4209119
:10288000E8002B772093E80008959091F300809161
:10289000F200089520919E01243019F08FEF9FEFF0
:1028A0000895FC014489558966897789452B462B13
:1028B000472BA1F386818F708093E9008091E80017
:1028C00082FFECCF9091F3008091F200892B79F098
:1028D0008091F10090E03091F3002091F200232BE1
:1028E00029F42091E8002B772093E80008958FEFDA
:1028F0009FEFF1CFA8E0B0E0E0E8F4E10C9484159C
:102900008C0180919E01843059F5F8018489958964
:10291000A689B789892B8A2B8B2B11F183858F7020
:102920008093E90088E0EAE2F1E0DE01119601908F
:102930000D928A95E1F750E040E068E070E0CE014A
:1029400001960E94550F50E040E062E070E0C8013F
:1029500042960E94550F8091E8008E778093E800A0
:102960002896E4E00C94A01508950895CF93DF9382
:10297000EC018091E80083FF10C028818091A301C1
:102980009091A4012817190641F48091A001813289
:10299000E9F030F4803209F44EC0DF91CF91089510
:1029A000823209F47BC08332C1F780919F0181326A
:1029B000A1F78091E800877F8093E8000E9495103E
:1029C0006091A101CE010E94B514E7CF80919F01D3
:1029D000813A19F78091E800877F8093E800809121
:1029E000E80080FFFCCF8C899D89AE89BF898093E8
:1029F000F100492F5A2F6B2F77274093F100AD013B
:102A0000662777274093F1008B2F9927AA27BB27AA
:102A10008093F100888D8093F100898D8093F1007F
:102A20008A8D8093F1008091E8008E778093E80092
:102A30000E949510B2CF80919F01813209F0ADCFF5
:102A40008091E800877F8093E8008091E80082FF12
:102A500020C03091F1002091F1009091F10080911F
:102A6000F1003C8B2D8B9E8B8F8B8091F100888F9A
:102A70008091F100898F8091F1008A8F8091E80028
:102A80008B778093E8000E949510CE010E94B414C9
:102A900084CF80919E018111D8CF7FCF80919F01FB
:102AA000813209F07ACF8091E800877F8093E80037
:102AB0000E9495108091A1019091A201998B888B21
:102AC000CE010E94B41469CF991B79E004C0991F0C
:102AD000961708F0961B881F7A95C9F78095089578
:102AE000EE0FFF1F0590F491E02D09942F923F9275
:102AF0004F925F926F927F928F929F92AF92BF920E
:102B0000CF92DF92EF92FF920F931F93CF93DF93B9
:102B1000CDB7DEB7CA1BDB0B0FB6F894DEBF0FBE16
:102B2000CDBF09942A88398848885F846E847D8463
:102B30008C849B84AA84B984C884DF80EE80FD8065
:102B40000C811B81AA81B981CE0FD11D0FB6F894DB
:102B5000DEBF0FBECDBFED010895FB01DC0104C057
:102B60008D910190801921F441505040C8F7881B85
:102B7000990B0895FB01DC0102C001900D924150B8
:102B80005040D8F70895F999FECF92BD81BDF89ACB
:102B9000992780B50895A8E1B0E042E050E00C9498
:102BA000F715262FF999FECF92BD81BDF89A0197AE
:102BB00000B4021639F01FBA20BD0FB6F894FA9A85
:102BC000F99A0FBE08950396272F0E94D2150E94EE
:102BD000D115252F0E94D215242F0C94D2150196C1
:102BE000272F0E94D2150C94D115DC01CB01FC01DA
:102BF000F999FECF06C0F2BDE1BDF89A319600B456
:102C00000D9241505040B8F70895F894FFCF9D12AF
:102C1000C512AE13C512AE13F8121913AE1370130A
:022C20007C1323
:102C22004F0101831000000104100000018208001E
:102C320000010000000000000000000000110D165D
:102C42000D430D140D440D150D01A12000000000CF
:0E2C5200020034C697669490F7313332360094
:00000001FF
